:020000040000FA
:04000000E6303A2884
:040004000034003490
:08000800A000030EA100831209
:1000100005191128831601178312B2308100B1012E
:100020002C2883160113831203140B190310A80D37
:10003000A90DAA0DAB0DAC0DAC16FF302C02031DA3
:100040002C28FA302B02031D2C2832152A08AF0069
:100050002908AE002808AD008B100B11210E83007B
:06006000A00E200E0900B5
:0C007400203084008001840A80300402E7
:10008000031C3C28152283160C308505870183123A
:10009000850187010730990000309A0010308316DF
:1000A0008E008312603083168F0083120030831617
:1000B000910000008312C830831681008312313012
:1000C0009000003083168C00831210308B003D238B
:1000D00081018E018F010B118B100B108C018B177E
:1000E0007F2032198B20B40B7D280310851903144F
:1000F000BA0DF0303A0203195E218423702864009F
:100100003310B10A311F8A28AC01AB01AA01A90141
:10011000A801B101080032110130B7008B13203063
:100120003707371A313E83169B001C141A088312B6
:10013000A40010303707371A313E83169B001C1479
:100140001A088312A300A6000230A6060030370763
:10015000371A313E83169B001C141A088312A20022
:10016000A7000130A7068B17331CBC2822090339CE
:10017000A200A309A409A50924082F02031D5829D8
:1001800023082E02031D582922082D02031D582979
:1001900001303702031DD1283E18D1283E143F14E8
:1001A000302202303702031DDA28BE18DA28BE14C6
:1001B0003F143C2203303702031DE3283E19E32895
:1001C0003E153F14482204303702031DEC28BE19A7
:1001D000EC28BE153F14542205303702031DF528C4
:1001E0003E1AF5283E163F14602206303702031DE2
:1001F000FE28BE1AFE28BE163F146C2207303702B6
:10020000031D07293E1B07293E173F14782208309B
:100210003702031D1029BE1B1029BE173F1484226C
:1002200009303702031D19295E1819295E143F147D
:1002300090220A303702031D2229DE182229DE14FB
:100240003F149B220B303702031D2B295E192B29EB
:100250005E153F14A6220C303702031D3429DE1927
:100260003429DE153F14B1220D303702031D3D291C
:100270005E1A3D295E163F14BC220E303702031D64
:100280004629DE1A4629DE163F14C7220F303702F0
:10029000031D4F295E1B4F295E173F14D2221030D9
:1002A0003702031D5829DE1B5829DE173F14DF22B1
:1002B000B70A11303702031808008E280130B60043
:1002C000B400B500B70085018701B2133A237F203F
:1002D000B40B7729031085190314BA0DF0303A02D4
:1002E0000319A529B50B77299630B500B121321D28
:1002F00067293211331C81292D090339AD00AE095C
:10030000AF092F1C67292D083002031967292D0812
:10031000B0002E1E67298B1320303707371A313E65
:10032000BC002F08BB00002210303707371A313EBF
:10033000BC002E08BB00002200303707371A313EC0
:10034000BC002D08BB0000228B1785018701B70A6E
:10035000B6010130B50011303702031C67293D2377
:100360000800013037020319EA220230370203196C
:10037000EF22033037020319F42204303702031945
:10038000F922053037020319FE220630370203191D
:1003900003230730370203190823083037020319F3
:1003A0000D2309303702031912230A3037020319CB
:1003B00017230B30370203191C230C3037020319A3
:1003C00021230D303702031926230E30370203197B
:1003D0002B230F3037020319302310303702031953
:1003E000352308003F1C08003F101030BC003E08B9
:1003F000BB0000223030BC005E08BB0000220800B9
:100400008B133B0883161C159A0083123C08831635
:100410009B0055309D00AA309D009C1464009C18E0
:100420000E2A1C1183128B170800831610309B00B4
:100430001C141A088312BE00831630309B001C1453
:100440001A088312DE00FF30C800CA15CB15CC1580
:10045000CD15CE15CF15D015D115D215D315080051
:100460000130BE05FF30DE050130C405C00000309C
:10047000C200C6005F1008000230BE05FF30DE0576
:100480000230C405C0000230C200C6005F10080080
:100490000430BE05FF30DE050230C405C000003068
:1004A000C200C6005F1008000830BE05FF30DE0540
:1004B0000A30C405C0000830C200C6005F10080042
:1004C0001030BE05FF30DE050A30C405C000003024
:1004D000C200C6005F1008002030BE05FF30DE05F8
:1004E0000430C405C0000430C200C6005F1008001C
:1004F0004030BE05FF30DE050C30C405C0000430BE
:10050000C200C6005F1008008030BE05FF30DE0567
:100510000430C405C0000030C200C6005F100800EF
:10052000FF30BE050130DE050830C505C1000030D2
:10053000C300C7000800FF30BE050230DE051030E2
:10054000C505C1001030C300C7000800FF30BE055C
:100550000430DE051030C505C1000030C300C700FF
:100560000800FF30BE050830DE055030C505C1006B
:100570004030C300C7000800FF30BE051030DE0564
:100580005030C505C1000030C300C7000800FF306F
:10059000BE052030DE052030C505C1002030C30077
:1005A000C70008000516FF30BE054030DE0560308C
:1005B000C505C1002030C300C70008000512FF3088
:1005C000BE058030DE052030C505C1000030C30007
:1005D000C70008001030850600308706080020306C
:1005E0008506003087060800203085060030870623
:1005F0000800223085060030870608002230850674
:1006000000308706080001308506003087060800A4
:10061000033085060030870608000130850600306B
:100620008706080000308506043087060800003081
:1006300085060130870608000030850601308706F0
:100640000800003085061130870608000030850656
:100650001130870608000030850620308706080024
:1006600000308506303087060800003085062030CF
:10067000870608003E18EA2208003E183022BE18FD
:100680003C223E194822BE1954223E1A6022BE1A4C
:100690006C223E1B7822BE1B84225E189022DE183C
:1006A0009B225E19A622DE19B1225E1ABC22DE1A36
:1006B000C7225E1BD222DE1BDF220800B601B40176
:1006C000B5013D1C662BBD01BD14682BBD013D1459
:1006D0003D08B60064006C2B6D2B6E2B6F2B702BBE
:1006E000FF30B51B8500B51F8501B40B6A2BB50B18
:1006F0006A2B0310B60CB608031D6A2B0030BC0031
:100700003D08BB00002208008F08031908008F0174
:1007100078308E00C80FAE2DC80A441CB42B461C7E
:10072000A52BCA1C962BCA014A15C22B4A1D9B2B0E
:10073000CA01CA15C22BCA1DA02BCA014A16C22B58
:100740004A1EC22BCA01CA14C22B4A1DAA2BCA01B7
:100750004A16C22BCA1DAF2BCA014A16C22B4A1E0B
:10076000C22BCA01CA14C22BCA1CB92BCA014A1512
:10077000C22B4A1DBE2BCA01CA15C22B4A1EC22B50
:10078000CA014A15C41CE92BC61CDA2BCB1CCB2B87
:10079000CB014B15F72B4B1DD02BCB01CB15F72BDA
:1007A000CB1DD52BCB014B16F72B4B1EF72BCB01BB
:1007B000CB14F72B4B1DDF2BCB014B16F72BCB1D8F
:1007C000E42BCB014B16F72B4B1EF72BCB01CB1495
:1007D000F72BCB1CEE2BCB014B15F72B4B1DF32B23
:1007E000CB01CB15F72B4B1EF72BCB014B15441D23
:1007F0001E2C461D0F2CCC1C002CCC014C152C2C77
:100800004C1D052CCC01CC152C2CCC1D0A2CCC015C
:100810004C162C2C4C1E2C2CCC01CC142C2C4C1DEE
:10082000142CCC014C162C2CCC1D192CCC014C16A4
:100830002C2C4C1E2C2CCC01CC142C2CCC1C232C62
:10084000CC014C152C2C4C1D282CCC01CC152C2C5F
:100850004C1E2C2CCC014C15C41D542CC61D452CF3
:10086000CD1C362CCD014D155F13622C4D1D3B2C3C
:10087000CD01CD15622CCD1D402CCD014D16622C25
:100880004D1E622CCD01CD14622C4D1D4A2CCD0184
:100890004D16622CCD1D4F2CCD014D16622C4D1ED8
:1008A000622CCD01CD14622CCD1C592CCD014D15DF
:1008B000622C4D1D5E2CCD01CD15622C4D1E622C7F
:1008C000CD014D155F1B8B2C441E8B2C461E7C2CA2
:1008D000CE1C6D2CCE014E15992C4E1D722CCE01C6
:1008E000CE15992CCE1D772CCE014E16992C4E1E6E
:1008F000992CCE01CE14992C4E1D812CCE014E1672
:10090000992CCE1D862CCE014E16992C4E1E992C5C
:10091000CE01CE14992CCE1C902CCE014E15992CC4
:100920004E1D952CCE01CE15992C4E1E992CCE0124
:100930004E15C51DC02CC71DB12CCF1CA22CCF013C
:100940004F15CE2C4F1DA72CCF01CF15CE2CCF1D70
:10095000AC2CCF014F16CE2C4F1ECE2CCF01CF1476
:10096000CE2C4F1DB62CCF014F16CE2CCF1DBB2C3D
:10097000CF014F16CE2C4F1ECE2CCF01CF14CE2C34
:10098000CF1CC52CCF014F15CE2C4F1DCA2CCF012B
:10099000CF15CE2C4F1ECE2CCF014F15451EF52C5A
:1009A000471EE62CD01CD72CD0015015032D501D0E
:1009B000DC2CD001D015032DD01DE12CD001501618
:1009C000032D501E032DD001D014032D501DEB2CF0
:1009D000D0015016032DD01DF02CD0015016032D40
:1009E000501E032DD001D014032DD01CFA2CD001A1
:1009F0005015032D501DFF2CD001D015032D501E76
:100A0000032DD0015015C51E2A2DC71E1B2DD11C2C
:100A10000C2DD1015115382D511D112DD101D1159C
:100A2000382DD11D162DD1015116382D511E382DBE
:100A3000D101D114382D511D202DD1015116382D41
:100A4000D11D252DD1015116382D511E382DD10122
:100A5000D114382DD11C2F2DD1015115382D511DF8
:100A6000342DD101D115382D511E382DD1015115FC
:100A7000451F602D471F512DD21C422DD20152150A
:100A8000DF136E2D521D472DD201D2156E2DD21DB2
:100A90004C2DD20152166E2D521E6E2DD201D21443
:100AA0006E2D521D562DD20152166E2DD21D5B2D6C
:100AB000D20152166E2D521E6E2DD201D2146E2D01
:100AC000D21C652DD20152156E2D521D6A2DD201F8
:100AD000D2156E2D521E6E2DD2015215DF1B972D91
:100AE000C51F972DC71F882DD31C792DD3015315F2
:100AF000A52D531D7E2DD301D315A52DD31D832DDB
:100B0000D3015316A52D531EA52DD301D314A52D06
:100B1000531D8D2DD3015316A52DD31D922DD30119
:100B20005316A52D531EA52DD301D314A52DD31CCB
:100B30009C2DD3015315A52D531DA12DD301D315E4
:100B4000A52D531EA52DD3015315F2214008C40035
:100B50004108C5005F18DF145F1CDF104808C9009A
:100B60000C304A05031D05120C304B05031D851280
:100B70000C304C05031D05100C304D05031D851070
:100B80000C304E05031D87100C304F05031D071157
:100B90000C305005031D07100C305105031D871242
:100BA0000C305205031D07120C305305031D87112D
:100BB00049080E020318082E12304A05031D0516B7
:100BC00012304B05031D851612304C05031D05140C
:100BD00012304D05031D851412304E05031D871478
:100BE00012304F05031D071512305005031D071461
:100BF00012305105031D871612305205031D0716CA
:100C000012305305031D8715FF30480203190800F1
:100C10008F08031D08007F2049080E02031C082EC0
:100C200018304A05031D051206304A05031D051636
:100C300018304B05031D851206304B05031D851624
:100C400018304C05031D051006304C05031D051416
:100C500018304D05031D851006304D05031D851404
:100C600018304E05031D871006304E05031D8714EE
:100C700018304F05031D071106304F05031D0715DA
:100C800018305005031D071006305005031D0714CA
:100C900018305105031D871206305105031D8716B4
:100CA00018305205031D071206305205031D0716A2
:100CB00018305305031D871106305305031D871592
:020CC00008002A
:084000000B00030007000100A2
:02400E00CC33B1
:10420000010078007A007C007E007B0079007F004E
:104210007D007A0078007E007C007D007F007900C0
:104220000100F200F600FA00FE00F200F600FA00CB
:10423000FE00F200F600FA00FE00F200F600FA00BE
:10424000FF00050005000500050009000900090040
:1042500009000D000D000D000D00110011001100EE
:104260000100FF00FF00FF00FF00FF00FF00FF0054
:10427000FF00FF00FF00FF00FF00FF00FF00FF0046
:10428000FF007B00FF00FF00FF00FF00FF00FF00BA
:10429000FF00FF00FF00FF00FF00FF00FF00FF0026
:1042A000FF00FE00FF00FF00FF00FF00FF00FF0017
:1042B000FF00FF00FF00FF00FF00FF00FF00FF0006
:1042C000FF001100FF00FF00FF00FF00FF00FF00E4
:1042D000FF00FF00FF00FF00FF00FF00FF00FF00E6
:1042E000FF00FF00FF00FF00FF00FF00FF00FF00D6
:1042F000FF00FF00FF00FF00FF00FF00FF00DD00E8
:00000001FF
